:1000000038C0A1C150C04FC04EC04DC04CC04BC045
:100010004AC04AC048C047C046C045C06AC143C084
:1000200042C041C040C053EF6E310000000053EFAA
:100030006E35000000004578697400000000200A59
:1000400052756E6E696E672054696D653A0A006874
:1000500028486F757229200068284D696E290A00AA
:100060006828486F757229200068284D696E290A32
:10007000000011241FBECFE5D4E0DEBFCDBF10E0ED
:10008000A0E6B0E0ECE8F9E102C005900D92A036E0
:10009000B107D9F712E0A0E6B0E001C01D92A13B84
:1000A000B107E1F75AC1ACCF1F920F920FB60F9272
:1000B00011242F933F934F935F936F937F938F936D
:1000C0009F93AF93BF93EF93FF9383EB82BF809196
:1000D0009B02882329F080919B02815080939B0290
:1000E0002091AD022223C9F480919E028F5F8093FC
:1000F0009E0280919E02843658F080919C029091DD
:100100009D028C5A91400CF4919820939E0205C058
:1001100080919E02823309F4919A809190028F5FC0
:1001200080939002809190028436E8F010929002C1
:100130008091A9028F5F8093A9028091A9028C33DC
:1001400090F01092A90280919A028F5F80939A0298
:1001500080919A028C3338F010929A028091B0020A
:100160008F5F8093B0029091A6021092A6029B9995
:1001700013C090FF0BC0809164008F5F8093640078
:1001800080916400882329F48FEF01C081E080937F
:10019000640081E08093A6029A9915C091FF0BC07C
:1001A0008091A8028F5F8093A8028091A802882383
:1001B00029F48FEF01C081E08093A8028091A6020C
:1001C00082608093A602999915C092FF0BC080911E
:1001D00095028F5F8093950280919502882329F480
:1001E0008FEF01C081E0809395028091A602846028
:1001F0008093A602989932C080919F028F5F80936E
:100200009F0280919F02882319F48FEF80939F02B1
:1002100080919F028431E0F08091A702885F8093F3
:10022000A7028091A702803D18F08FEC8093A7026F
:100230008091A7029927382F22278091A70299271A
:10024000282B392BB9018BE0F6D981E080939F02EE
:100250008091A60288608093A60202C010929F023D
:10026000B09932C08091AA028F5F8093AA028091D8
:10027000AA02882319F48FEF8093AA028091AA0220
:100280008431E0F08091A70288508093A70280918A
:10029000A7028F3F19F487E08093A7028091A702FD
:1002A0009927382F22278091A7029927282B392BAD
:1002B000B9018BE0C0D981E08093AA028091A602A7
:1002C00080618093A60202C01092AA028EEC86B9C9
:1002D000FF91EF91BF91AF919F918F917F916F911E
:1002E0005F914F913F912F910F900FBE0F901F90F4
:1002F00018951F920F920FB60F9211242F933F93D0
:100300008F939F9384B1282F332785B199278370CA
:100310009070982F882790939D0280939C028091E3
:100320009C0290919D02822B932B90939D0280932F
:100330009C0237989F918F913F912F910F900FBE04
:100340000F901F9018951F920F920FB60F921124C5
:100350000F900FBE0F901F901895CFE5D4E0DEBF31
:10036000CDBF8DE088BB8EE287BB8FE085BB80E18F
:1003700084BBC1E0C2BB88EF81BB04B603FE02C0F0
:100380008C2F63D814BE9B9B09C0C093AD0210BCD8
:1003900098E199B980E28BB99AB904C01092AD0284
:1003A000899A919AA89588E181BD8FE181BD85ECFC
:1003B00087B983EB82BF85E083BF89B7816089BF3E
:1003C00083E885BF1092A60210929D0210929C02B3
:1003D00010929102789480919C0290919D028A598A
:1003E000914044F4889580919C0290919D028A5995
:1003F0009140C4F3AC9A88E280939B028CE0B8D819
:100400008093A7028091A7028F3F19F487E480931D
:10041000A70281E0ADD899279093A1028093A00212
:1004200083E0A6D89927982F882790936702809316
:10043000660282E09DD8282F332780916602909132
:100440006702822B932B909367028093660286E06B
:100450008FD89927AA27BB27DC0199278827809363
:10046000960290939702A0939802B093990285E028
:100470007FD89927AA27BB272227382F492F5A2F01
:100480008091960290919702A0919802B091990262
:10049000822B932BA42BB52B8093960290939702DB
:1004A000A0939802B093990284E062D8282F332752
:1004B000442755278091960290919702A091980227
:1004C000B0919902822B932BA42BB52B809396028B
:1004D00090939702A0939802B09399028BE048D82A
:1004E0009927AA27BB27B82FAA279927882780935F
:1004F0008A0290938B02A0938C02B0938D028AE0C3
:1005000037D89927AA27BB27AC0133272227809108
:100510008A0290918B02A0918C02B0918D02822B65
:10052000932BA42BB52B80938A0290938B02A093DC
:100530008C02B0938D0289E01BD89927AA27BB278C
:100540002227382F492F5A2F80918A0290918B02AF
:10055000A0918C02B0918D02822B932BA42BB52BF2
:1005600080938A0290938B02A0938C02B0938D02A9
:1005700088E0FED7282F33274427552780918A0209
:1005800090918B02A0918C02B0918D02822B932BC3
:10059000A42BB52B80938A0290938B02A0938C029C
:1005A000B0938D02109290021092A9028EE0E0D7D3
:1005B00080939A028DE0DCD78093B00280919A02FA
:1005C0008F3F21F410929A021092B0028091AD02F6
:1005D0008823D9F08EE390E07AD98091B00262D975
:1005E0008FE490E074D980919A025CD988E590E01C
:1005F0006ED98FE0BDD756D980E690E068D980E10A
:10060000B7D750D989E690E062D98091A60281FFE0
:1006100004C0109267021092660237D18F3F79F4BE
:1006200080919B02882329F0889580919B028823E2
:10063000D9F7C19A61E083E0A3D781E006D7809122
:100640009B02882329F0889580919B028823D9F703
:10065000C19AA89560E081E093D74BD1882329F017
:1006600061E082E08DD781E0F0D68FEF9FEF3BD243
:100670009093690280936802892B29F461E0862FA8
:100680007FD781E0E2D68091A0029091A102892BD0
:1006900031F481E090E09093A1028093A0028091D8
:1006A000A0029091A1021FD26091860280918702E0
:1006B0009927AA27BB272227382F492F5A2F260FE1
:1006C000311D411D511D809188029927AA27BB2702
:1006D000DC0199278827280F391F4A1F5B1F80914B
:1006E00089029927AA27BB27B82FAA2799278827E5
:1006F000280F391F4A1F5B1F80918A0290918B023D
:10070000A0918C02B0918D0282179307A407B507C0
:1007100051F081E090E09093A1028093A0021092AA
:100720006702109266022091A0023091A10280918E
:100730006802909169028217930730F481E090E09B
:100740009093A1028093A0028BD080919602909109
:100750009702A0919802B09199029C01AD0160911D
:100760006602709167028091A0029091A1025CD212
:10077000C82F76D0C7FF05C0C19561E08C2F00D788
:1007800036C0C130B9F580916400853680F1809122
:100790009C0290919D028D5F914014F060E025C015
:1007A00080919C0290919D02895E914014F060E0DE
:1007B00019C080919C0290919D02855D914014F03A
:1007C00060E04BC080919C0290919D02815C9140C1
:1007D0000CF042C080919C0290919D028D5A9140F4
:1007E0001CF06C2F82E03AC06C2F83E037C080E0B1
:1007F0002CD62AC0C330D9F48091A802853618F0CF
:1008000081E090E019C08091A8028A31C8F08091FF
:10081000A0029091A10201979093A1028093A0025F
:10082000892B71F4809168029091690205C08091D2
:10083000A0029091A10201969093A1028093A00240
:10084000109267021092660280919C0290919D0224
:100850008A5991400CF067CF61E081E091D663CF77
:100860007894A895889588958091A6029927877095
:100870009070892BB1F7889588958091A602992769
:1008800087709070892B69F70895CF9382E58DB9B1
:10089000C29AC0E0CAD7CF5FCA30E0F3C29840E046
:1008A00050E060E070E080E078D7C82F813071F0D0
:1008B0008F3F61F0889540E050E060E070E080E0BC
:1008C0006CD7C82F813011F08F3FA1F7C13049F4A8
:1008D00040E050E060E070E081E05FD7C82F8130F9
:1008E000B9F3C29A80E58DB9709A8C2F9927CF9170
:1008F0000895EF92FF920F931F93CF93DF936EEBC8
:1009000071E080E090E0B9D620917202809173028C
:100910009927D82FCC27C20FD11D7E010027112780
:1009200049E0EE0CFF1C001F111F4A95D1F7C801CA
:10093000B701A3D620917502809176029927982F4E
:100940008827820F911D8050924019F082E090E03C
:10095000C3C0809177028093650080917802FE0188
:10096000E80FF11D809179029927982F8827E80FC9
:10097000F91FF093AC02E093AB0220917B028091CF
:100980007C029927782F6627620F711D7093AF0242
:100990006093AE0220918002809181029927582FA6
:1009A0004427420F511D4115510519F481E090E093
:1009B00093C080917A029927849FE001859FD00D92
:1009C000949FD00D1124CE018E0F9F1F90939402FF
:1009D00080939302AB01A4E056954795AA95E1F761
:1009E0006F707070672B11F04F5F5F4FAA27BB27A6
:1009F000EA01EE27FF278C0F9D1FAE1FBF1F8093BC
:100A0000600090936100A0936200B0936300209116
:100A10007D0280917E029927AA27BB27FA2FE92F12
:100A2000D82FCC27C20FD11DE11DF11D2097E10564
:100A3000F10581F5D801C7018096A11DB11DBC014A
:100A4000CD011BD620916A0280916B029927AA27BB
:100A5000BB27FA2FE92FD82FCC27C20FD11DE11DBC
:100A6000F11D80916C029927AA27BB27DC019927E9
:100A70008827C80FD91FEA1FFB1F80916D02992795
:100A8000AA27BB27B82FAA2799278827C80FD91FBD
:100A9000EA1FFB1F8091AB029091AC02AA27BB27F3
:100AA000C81BD90BEA0BFB0B80916500282F33275D
:100AB00044275527BE01CF0147D7FA01E901C050AD
:100AC000D041E040F04020F081E08093920202C0EB
:100AD0001092920280E090E0DF91CF911F910F91F0
:100AE000FF90EF9008954F925F926F927F928F9256
:100AF0009F92BF92CF92DF92EF92FF920F931F933C
:100B0000CF934C01662477248091930290919402B4
:100B10007C010027112779E0EE0CFF1C001F111F3C
:100B20007A95D1F723018091AE029091AF026816B9
:100B3000790608F069C0C801B701E3D5882309F038
:100B400063C0B82EC0E06AE6C62E62E0D62E6DD62F
:100B5000D6018D936D01CF5FC032C8F390916A02C8
:100B6000992369F180918402882321F48091850280
:100B70008823F1F0953EE1F0809175029927887104
:100B80009070892BA9F4809172028D3489F4809140
:100B90007302803569F480917402833349F40894B8
:100BA000611C711C0894810891088114910439F02A
:100BB0000894411C511CB394BFE0BB1518F6B394C4
:100BC000EFE0EB1548F0C0E030D6CF5FC032E0F385
:100BD000B394FFE0FB15B8F7CED580916A02882365
:100BE00099F08114910481F080E092E0A0E0B0E0FF
:100BF000E80EF91E0A1F1B1F8091AE029091AF02F2
:100C00004816590608F497CFC301CF911F910F9151
:100C1000FF90EF90DF90CF90BF909F908F907F904C
:100C20006F905F904F900895AF92BF92CF92DF92F6
:100C3000EF92FF920F931F93CF93DF938C01EB0101
:100C400069017A0150DF0817190719F08FEF9FEF3C
:100C500026C220918602809187029927AA27BB2766
:100C60004427582F692F7A2F420F511D611D711D86
:100C7000809188029927AA27BB27DC01992788271A
:100C8000480F591F6A1F7B1F809189029927AA2745
:100C9000BB27B82FAA2799278827480F591F6A1FF3
:100CA0007B1F40938A0250938B0260938C02709357
:100CB0008D022097D1F0D0936702C0936602C09254
:100CC0009602D0929702E0929802F092990209E07F
:100CD000CC0CDD1CEE1CFF1C0A95D1F7A0908A02FB
:100CE000B0908B02AC18BD0822C020918402809184
:100CF00085029927982F8827820F911D909367026C
:100D000080936602DB01CA01C9E0B695A795979565
:100D10008795CA95D1F78093960290939702A093F6
:100D20009802B09399025170607070705A0180916E
:100D30006602909167022FEF8F3F920709F45EC120
:100D40008230910508F45AC120E030E040E050E0E4
:100D500060E070E0AFD190938F0280938E0210928A
:100D600064001092A8021092950220916500C22F93
:100D7000DD278091660290916702AA27BB27029720
:100D8000A109B109332744275527BC01CD01BDD5A1
:100D90006B017C018091600090916100A0916200E4
:100DA000B0916300C80ED91EEA1EFB1EB9E0CC0C40
:100DB000DD1CEE1CFF1CBA95D1F708D484E68093A5
:100DC0009B028091960290919702A0919802B09117
:100DD0009902181619061A061B060CF002C1C70163
:100DE000B6018FD4882309F009C1F8948FEF19D583
:100DF00000E010E082991CC0A89584E680939B02D5
:100E000080918E0290918F02892B69F49801B7012D
:100E1000A60180916602909167024CD190938F0257
:100E200080938E0203C078948895F894829BE4CFD7
:100E30009FB18FEF8FB997FF02C0979A01C0979823
:100E4000949A939A990F9398949886E097FF02C08A
:100E5000979A01C09798939A990F9398815087FF1A
:100E6000F5CF0F5F1F4F82E00030180708F4C2CFA4
:100E7000789481D48091960290919702A0919802E3
:100E8000B09199020197A109B109809396029093BC
:100E90009702A0939802B0939902219749F180E0BC
:100EA00092E0A0E0B0E0C80ED91EEA1EFB1E8091C1
:100EB000AD02882309F46CC0C130D10509F068C0C7
:100EC00000919C0210919D02812F9927EBD4802FD5
:100ED000E9D480E2E3D48091660290916702892F81
:100EE0009927E0D480916602DDD48AE0D7D450C03F
:100EF00080918E0290918F02009779F49E0140E0DC
:100F000050E060E070E08091660290916702D2D07C
:100F1000909367028093660208C090936702809363
:100F20006602D0938F02C0938E02809166029091E8
:100F30006702AFEF8F3F9A0719F08230910518F4DE
:100F4000AA24BB244EC0AA27BB270297A109B10936
:100F500010916500212F332744275527BC01CD016F
:100F6000D4D46B017C018091600090916100A091CC
:100F70006200B0916300C80ED91EEA1EFB1EE9E0B4
:100F8000CC0CDD1CEE1CFF1CEA95D1F7C12FDD2730
:100F900039D210919B02112351F4809191021816BD
:100FA00084F181E0809391021093A80247C0809160
:100FB0006400833070F580919502833090F58091C4
:100FC000A8028330B0F58091960290919702A0918B
:100FD0009802B0919902181619061A061B060CF40D
:100FE000FECE10929102C50101978F5F914008F0EB
:100FF00054C0C701B60185D3882319F18EEF9FEF46
:101000004EC061E0862FBCD21093910210939502DE
:101010000DC060E081E0B4D21092910281E090E0D6
:101020003EC060E081E0ACD21092910282E090E09C
:1010300036C060E081E0A4D21092910283E090E09B
:101040002EC0F8948FEFEDD300E010E02FB18FEFBA
:101050008FB9C5010894A108B108892BB1F0829914
:1010600006C0A89578948895F894829BFACF949AB4
:1010700087E027FF02C0979A01C09798939A220FA2
:1010800093989498815087FFF4CF0F5F1F4F22E011
:1010900000301207D8F278946ED380E090E0DF91B0
:1010A000CF911F910F91FF90EF90DF90CF90BF9065
:1010B000AF9008954F925F926F927F928F929F921E
:1010C000AF92BF92CF92DF92EF92FF920F931F9356
:1010D000CF93DF932C014A015B0139018091920289
:1010E0006091AB027091AC0292014427552788238E
:1010F00009F0C3C07B0100271127C9E0EE0CFF1CDB
:10110000001F111FCA95D1F7E20EF31E041F151F11
:10111000C20196958795AA27BB27E80EF91E0A1FDC
:101120001B1FD801C7019170A070B0708F5F9140F4
:10113000A040B04009F04CC081149104A104B10456
:1011400099F1E30180E0681682E0780630F46DD30F
:10115000219622E0C030D207D0F30DD3C801B701E9
:10116000F4D06C018FEFC822DD240894E11CF11C3F
:10117000011D111DC801B701E8D0982F8827C82A82
:10118000D92AC501B401BDD2882309F0B1C04DD31D
:10119000C0E0D0E0C615D70508F059C046D3219667
:1011A000C615D705D8F353C0C801B701CED06C011E
:1011B0002FEFC222DD240894E11CF11C011D111D3A
:1011C000C801B701C2D0982F8827C82AD92A3FC0A2
:1011D000A801970120703E7F81149104A104B104FD
:1011E00091F18091A2029091A302A091A402B091EA
:1011F000A502281739074A075B0729F1E30180E0B8
:10120000681682E0780630F410D3219622E0C030D0
:10121000D207D0F3B0D2C801B70197D06C01C50195
:10122000B4016FD2882319F08FEF9FEF7DC0FDD2FC
:10123000C0E0D0E0C615D70550F4F7D22196C61508
:10124000D705D8F304C0C801B7017FD06C0140FEB8
:1012500007C02601E4E056944794EA95E1F706C0FA
:101260007FEF472E7FE0572E4C205D2088EF4816F9
:101270008FE0580608F457C053C0CB01AA27BB27FC
:10128000EE24F82E092F1A2FE20EF31E041F151F4D
:10129000EE0CFF1C001F111FA801970120703E7F5C
:1012A00081149104A104B10491F18091A202909162
:1012B000A302A091A402B091A502281739074A07FA
:1012C0005B0729F1E30120E0621622E0720630F4A8
:1012D000ACD2219682E0C030D807D0F34CD2C801FE
:1012E000B70133D02C01C501B4010BD2882319F00A
:1012F00080E090E019C099D2C0E0D0E0C615D705D3
:1013000050F493D22196C615D705D8F304C0C8016E
:10131000B7011BD02C0128EF42162FEF520618F010
:101320005FEF452E552EC201DF91CF911F910F9196
:10133000FF90EF90DF90CF90BF90AF909F908F90F5
:101340007F906F905F904F900895CF92DF92EF92D1
:10135000FF920F931F93CF93DF937B018C018FEF4D
:10136000C82E81E0D82ECE20DF2080E09EEFAFEFA8
:10137000BFEFE822F9220A231B238091A202909159
:10138000A302A091A402B091A502E816F9060A07EB
:101390001B07E9F0C801B701B4D1882319F020E098
:1013A00030E026C0C6E6D0E092E0C636D90730F479
:1013B0003CD28993A2E0C636DA07D0F3DCD1E092C2
:1013C000A202F092A3020093A4021093A502F601D8
:1013D000EA59FF4F8081282F3327E7E6F0E0CE0E51
:1013E000DF1ED6018C919927982F8827282B392B1F
:1013F000C901DF91CF911F910F91FF90EF90DF9086
:10140000CF90089580919C0290919D028C579140BD
:10141000BCF4C29A61E084E0B3D0F8948091B00249
:10142000882361F060919A0280E191D06091B002CE
:101430008FE08DD010929A021092B00280E005D019
:1014400080919C0290919D0208951F93182FF8940B
:10145000C29AC19860E170E080E0EDD0112309F0FC
:1014600072C06091A7028CE072D06091A00281E00E
:101470006ED06091660282E06AD08091660290919F
:101480006702892F9927682F83E061D060919602C7
:1014900084E05DD08091960290919702A09198028D
:1014A000B0919902892F9A2FAB2FBB27A7FDBA9530
:1014B000682F85E04CD08091960290919702A09180
:1014C0009802B0919902CD01BB2797FDB095AB2F43
:1014D000682F86E03CD060918A0288E038D0809105
:1014E0008A0290918B02A0918C02B0918D02892F7B
:1014F0009A2FAB2FBB27682F89E029D080918A02D1
:1015000090918B02A0918C02B0918D02CD01AA27FF
:10151000BB27682F8AE01BD080918A0290918B02B2
:10152000A0918C02B0918D028B2F9927AA27BB27FF
:10153000682F8BE00CD060919A028EE008D0609109
:10154000B0028DE004D0AC98A8958895FCCF1F938D
:10155000CF93C82F162F0CD0811739F0E199FECF09
:101560001FBACEBB1DBBE29AE19ACF911F9108959D
:10157000E199FECF1FBA8EBBE09A8DB399270895EB
:101580001F93CF93C82F162FF89420D07894CC2394
:10159000B9F0112319F08EE290E002C086E290E0EB
:1015A00033D083E18895815087FFFCCF86E390E0BC
:1015B0002BD085E08895815087FFFCCFC15049F73B
:1015C00086E390E021D0CF911F91089564E070E010
:1015D00080E031D090D060E070E080E02CD0829B41
:1015E000FECF8091A7029927382F22278091A7024A
:1015F0009927282B392BB9018BE01DD067EF7BE9A8
:1016000083E019D078D0089540E0FC010196249140
:10161000949A30E027FF02C0979A01C09798939A56
:10162000220F939894983F5F3830A0F3979A4F5FBA
:10163000483058F30895FF920F931F93F82E8B01B3
:10164000959882E00CD08F2D0AD0812F992707D052
:10165000802F05D0959A1F910F91FF90089597E0E4
:1016600087FF02C0979A01C09798969A880F96981C
:10167000915097FFF5CF979A0895CF92DF92EF920E
:10168000FF920F931F93CF93DF937B018C01DC01BB
:10169000CB0180709E7FBC01CD0133D0882311F532
:1016A000BFEFCB2EB1E0DB2ECE20DF2000E010E03C
:1016B0000C151D0579F4CAE6D2E0AFE1EA2EF12C53
:1016C000EC0EFD1EB2D089930F5F1F4FEC16FD0686
:1016D000CCF701C0AAD00F5F1F4F82E0003018077F
:1016E00038F349D0DF91CF911F910F91FF90EF9088
:1016F000DF90CF90089580E000008F5F8F3FE1F78B
:101700000895DF92EF92FF920F931F93CF93DF9391
:101710007B018C01DD24C298B801A70181E13DD095
:10172000982F882361F4C0E0D0E07FD0982F8E3FBF
:1017300041F0219687E0C03DD807B8F305C08E3F41
:1017400019F480E090E00FC0C29A8091AD02882326
:1017500021F0892FA7D080E2A1D0D39483E68D1504
:10176000D0F681E090E0DF91CF911F910F91FF9033
:10177000EF90DF900895CF93DF9357D056D0C0E01D
:10178000D0E053D08F3F29F0219683E0C83ED807A0
:10179000C0F3C29ADF91CF910895DF92EF92FF924A
:1017A0000F931F93CF93DF93D82E7A018B01C0E064
:1017B000D0E03BD08F3F29F0219693E0C83ED90777
:1017C000C0F38F3F19F081E090E023C080E4D82A75
:1017D0008D2D27D0812F9927AA27BB2722D0C8017A
:1017E000AA27BB271ED0BB27A12F902F8F2D19D042
:1017F0008E2D17D085E915D0C0E0D0E016D08E3FF1
:1018000039F088232CF4219693E0C83ED907B0F331
:101810009927DF91CF911F910F91FF90EF90DF906B
:1018200008958FB9779BFECF08958FEF8FB9779B7F
:10183000FECF8FB199270895779BFECF0895CF9360
:10184000DF93DC01CB0129E0880F991FAA1FBB1F82
:101850002A95D1F7BC01CD0154DF24D08AE01ED0F7
:10186000C0E0D0E0E2DF1ED0CE018F7190704F97C4
:1018700011F48AE003C0C0FF02C080E20FD02196BD
:1018800082E0C030D80774F376DFDF91CF910895FE
:10189000A8955F9BFDCF8CB1992708955D9BFECFE6
:1018A0008CB90895CF93C82F982F92959F70892F48
:1018B000805D8A3308F0895FF1DF9C2F9F70892F4C
:1018C000805D8A3308F0895FE9DFCF910895CF9377
:1018D000DF93EC01FC0121968491882331F0DEDF57
:1018E000FE01219684918823D1F7DF91CF9108954D
:1018F000CF93DF93EC018991882321F0CFDF899189
:101900008823E1F7DF91CF910895629FD001739F03
:10191000F001829FE00DF11D649FE00DF11D929F8B
:10192000F00D839FF00D749FF00D659FF00D9927CA
:10193000729FB00DE11DF91F639FB00DE11DF91FEE
:10194000BD01CF0111240895A1E21A2EAA1BBB1BD1
:10195000FD010DC0AA1FBB1FEE1FFF1FA217B3077B
:10196000E407F50720F0A21BB30BE40BF50B661F91
:10197000771F881F991F1A9469F760957095809555
:0C19800090959B01AC01BD01CF010895C2
:00000001FF
